:020000040800F2
:10000000680A002045410008A5160008A916000846
:10001000AD160008B1160008B51600080000000073
:10002000000000000000000000000000B9160008F9
:10003000BD16000800000000C11600089915000850
:100040005F4100085F4100085F4100085F41000810
:100050005F4100085F4100085F4100085F41000800
:100060005F410008211600084116000861160008CB
:100070005F410008051600085F4100085F41000865
:100080005F4100085F41000800000000B91500084A
:100090005F4100085F4100085F4100085F410008C0
:1000A0005F4100085F4100085F4100085F410008B0
:1000B0005F410008000000005F41000800000000F0
:1000C0005F410008000000005F4100085F41000838
:1000D0005F4100085F4100085F4100080000000028
:1000E00000000000000000005F4100085F410008C0
:1000F0005F4100085F4100085F4100085F41000860
:100100005F41000800000000000000005F4100089F
:1001100000000000000000000000000000000000DF
:1001200000000000000000000000000000000000CF
:1001300000000000000000000000000000000000BF
:1001400000000000000000000000000000000000AF
:1001500000000000000000005F4100085F4100084F
:100160005F4100085F41000800F002F800F03AF833
:100170000AA090E8000C82448344AAF10107DA4502
:1001800001D100F02FF8AFF2090EBAE80F0013F01A
:10019000010F18BFFB1A43F001031847BC560000BB
:1001A000DC560000103A24BF78C878C1FAD852074C
:1001B00024BF30C830C144BF04680C6070470000E1
:1001C0000023002400250026103A28BF78C1FBD860
:1001D000520728BF30C148BF0B6070471FB51FBD15
:1001E00010B510BD04F06FF81146FFF7F7FF00F0EF
:1001F00009F804F08DF803B4FFF7F2FF03BC04F034
:1002000095F8000004F01CF840F20000C2F2000073
:10021000006844F6D351C1F26201A0FB01014FF026
:10022000FF3000EB91110020B0EB116F0DD14EF2B9
:100230001002CEF2000251604EF62351CEF20001C0
:10024000F0230B7090600720106000F0ADFD0028D7
:1002500042D040F20044C4F6000400F0A1FD00F0DA
:10026000BFFD00F0EBFD4FF090400221012202F0B3
:100270000DF920460421012202F008F94FF49640BE
:1002800001F0FEF800F0F6FF00F03CFF02F028F865
:1002900040F27A180824C2F2000800BF642088F8EF
:1002A000004065B201F0F0F9002DA4F10104F5DC85
:1002B000002088F8000040F20040C4F6000000F57D
:1002C000806900BF48464FF4004102F0E7F820B1D2
:1002D00002F006F8F6E700BFFEE70A2001F0D4F9C5
:1002E0004FF090400221002202F0D0F840F2E815D1
:1002F00040F2102A40F2000BC2F20005C2F2000ADE
:10030000CCF27A4B01F0BAF929688842FAD301F0AD
:10031000B5F9DAF8001048F21F520131C5F2EB12BC
:10032000A1FB0223053028609809C82200FB1210A7
:10033000CAF8001064284FF0000248464FF40051FC
:1003400038BF012202F0A2F89AF80000C00708BFE7
:1003500001F0B8F940F20420C2F20000066830460D
:10036000002E48BF704204F023FF04F021FD00235B
:100370000022CBF6E073002704F02EFB44F20003CA
:100380000022C4F28F0304F0BFF800230022C3F65A
:10039000F07304F005F803F0D1FF06F13101632991
:1003A00004460DD340F20C00C2F20000B0F9000088
:1003B00041428E42C8BF31468642C8BF01464F42C5
:1003C00040F20C20C2F20000016801F13100632804
:1003D00002D2002013E000BF40F20C00C2F2000085
:1003E000B0F9002050428142C8BF08469142C8BFC0
:1003F000104604F0DDFE0146204604F06DFF04F0D7
:10040000BBFE04F0D5FE0146584605F031F8002445
:10041000C4F23434214604F05FFF0021C4F2FA41F3
:1004200004F0B4FD214604F0EFFC064604F0A4FEFF
:1004300045F28451C0F6000151F8204000213046B9
:10044000C4F2B42104F08FFD5E460FFA87FB1BF562
:100450007A7F4FF61841CFF6FF71D8BF8B46BBF5B8
:100460007A7FA8BF4FF47A7B10B3584604F0A0FE01
:100470000146204604F030FF3146044604F073FD87
:100480000026C4F27A4600281CBF0024CCF27A442D
:100490002046314604F067FD002808BF3446204658
:1004A00004F06AFE40F2FC11C2F20001088022E072
:1004B00040F2FC10C2F20000A0F800B0584604F070
:1004C00077FE214604F062FD3146044604F04BFD00
:1004D0000026C4F27A4600281CBF0024CCF27A44DD
:1004E0002046314604F03FFD002808BF3446204630
:1004F00004F042FE83460FFA8BF4204600F026FA01
:1005000040F20400C2F20000066800213046C4F246
:10051000A81104F021FDC8B940F20800C2F20000A1
:10052000007840F20421C2F2000101380968B0FAF3
:1005300080F0400911F1320F4FF00001B8BF0121E6
:10054000084001461CBF052104203CE030464F46D0
:10055000D14604F02DFC4CF6CC434FF0CC32C4F223
:10056000330380468A4604F0CDFC40B90021304672
:10057000C4F2A81104F0F7FC08B108201CE049F609
:100580009A1249F6991340465146C9F69912C4F297
:10059000320304F0B7FC002840F0E7804CF6CC436F
:1005A000404651464FF0CC32C4F2330304F0B1FC64
:1005B000002800F0DA80012040F27A180521C2F20A
:1005C0000008CA46B94688F8001040F27B11C2F212
:1005D0000001087048464FF4004101F05FFF002819
:1005E00062D18BEAE430A0EBE43080B2322805D946
:1005F00040F2000B0020CCF27A4B18E040F2FC10E5
:10060000C2F20000008840F2000B01B280EAE13043
:10061000A0EBE13080B23228CCF27A4B06D840F21F
:10062000EC10C2F200000068013000E0002043F648
:100630008101C0F20101884240F2EC11C2F20001D6
:10064000086056D240F20E00C2F200000078400668
:1006500005D540F2CC110020C2F20001087040F232
:10066000CC10C2F20000007800F06AF940F20E04EB
:10067000C2F2000420780221C0F3C0024FF0904083
:1006800001F004FF20780121C0F300124FF09040E8
:1006900001F0FCFE94F90000B0F1FF3F47DD01F0EE
:1006A0001FFE2FE601F01CFE48464FF4004101F00A
:1006B000F5FE0028F6D10024642088F8004000F000
:1006C000E3FF082C04F10104F6D3002088F80000B1
:1006D000002000F035F9002000F038F940F2004029
:1006E000C4F600000421002201F0D0FE01F0F8FD64
:1006F000FCE70024642088F8004000F0C5FF082CC7
:1007000004F10104F6D3002088F80000002000F076
:1007100017F9002000F01AF940F20040C4F600007A
:100720000421002201F0B2FE01F0DAFDFCE7002412
:10073000642088F8004000F0A7FF082C04F10104B1
:10074000F6D3002088F80000002000F0F9F800201F
:1007500000F0FCF840F20040C4F600000421002242
:1007600001F094FE01F0BCFDFCE749F69A1249F64F
:100770009913C9F69912C4F232034046514604F067
:10078000C8FB40F27A170024C2F20007E0B100BFB4
:1007900064203C7000F078FF082C04F10104F7D3CA
:1007A00000203870002000F0CBF8002000F0CEF8D8
:1007B00040F20040C4F600000421002201F066FE71
:1007C00001F08EFDFCE700BF64203C7000F05CFF90
:1007D000082C04F10104F7D300203870002000F049
:1007E000AFF8002000F0B2F840F20040C4F600007C
:1007F0000421002201F04AFE01F072FDFCE700BF77
:10080000704700BF40F20421C2F2000101380968BC
:10081000B0FA80F04009002211F1320FB8BF012276
:100820001040014640F27A121CBF05210420C2F29A
:100830000002117040F27B11C2F200010870704793
:1008400040F27A140025C2F2000400BF6420257033
:1008500000F01AFF082D05F10105F7D300202070E4
:10086000002000F06DF8002000F070F840F2004029
:10087000C4F600000421002201F008FE01F030FD62
:10088000FCE7000090FBF1F202FB1100084490FB32
:10089000F1F202FB110000B2704700BF401A4AF6A5
:1008A000AB2100B2C2F6AA2180FB012303EBD37275
:1008B00002EB4202A0EB4200063080FB011202EB89
:1008C000D27101EB4101A0EB410045F25A51C0F653
:1008D000000131F91000704780B5DDF808C0A1F1C2
:1008E000010EBEF1050F08D8DFE80EF0030D10145D
:1008F0001B220021116018601DE0002010601860AC
:10090000CCF8000080BD414211600CE04142116012
:10091000002102E00021116041421960CCF8000082
:1009200080BD1060404218600020CCF8000080BDFF
:100930000021106019604042CCF8000080BD00BF6B
:1009400040F27511C2F2000108707047F0B581B035
:1009500003F09FFF0023C3F6F273002204F03CF87B
:1009600049F20043CCF29103002205460C4604F004
:10097000D0FA49F20046C4F2910600281EBF49F29F
:100980000044CCF29104002528462146002233463B
:1009900004F0BFFA0746284621460022334604F0F9
:1009A000B8FA002808BF3446002F08BF3D46284645
:1009B000214603F03FFF40F27611C2F200010880A9
:1009C00001B0F0BD2DE9F04F81B040F2F810C2F255
:1009D0000000B0F90010B1F57A7F14DA40F270121D
:1009E00040F20A03C2F20002C2F200035288B3F9D5
:1009F000007001310180B81800EBD07040081880F9
:100A000001B0BDE8F08F40F27C1AC2F2000ABAF8D9
:100A1000004045F62940604381B2890841EA8030B0
:100A200080B2000940F270182828C2F2000834D8B9
:100A300040F2040BC2F2000BDBF8000004F0B8F93E
:100A40008146B8F800000D4603F03AFF4CF200036F
:100A5000C3F69873002203F0BFFF4AF6FC1246F279
:100A60004D23CDF2F122C3F6507303F0B5FF48F2E7
:100A70002B724FF2CE7306460F46CDF61612C3F612
:100A8000EF734846294603F0A7FF32463B4603F082
:100A900087FC03F053FCCBF8000040F27A10C2F25E
:100AA0000000007840F20045C4F60005611CAAF879
:100AB0000010A8B141F2597289B2CDF2B712A1FB70
:100AC000022340F27B12C2F2000212781F0B0132A5
:100AD000B7FBF2F77A43C2EB1332002A00F0AF8083
:100AE000002228464FF4806101F0D0FC40F20A0158
:100AF000C2F20001B8F80200B1F9001042F6004855
:100B0000401AC4F2010803F0C4FE48F23F024CF65A
:100B10009C13C9F6C912C3F6C97303F05DFF03F055
:100B20000DFC40F2801120F00040C2F2000108608C
:100B30000021C4F2701104F001FA80B940F275107E
:100B4000C2F20000007850B140F21420C2F200005E
:100B50000078012803D0404602F0E8FA02E040465F
:100B600002F0EAFA28464FF4006101F097FC40F2E7
:100B7000D516C2F20006307005F58050022101F052
:100B80008DFC40F2D617C2F20007387005F5806080
:100B90004FF4804101F082FC40F2D714C2F200040D
:100BA000327820704FF090404FF4004101F06EFC1D
:100BB0003A784FF090404FF4805101F067FC227872
:100BC0002846082101F062FC30783978227800EB61
:100BD000410040F2D41100EB8200C2F20001087023
:100BE00045F27A5140F2D012C0B2C0F60001C2F212
:100BF000000240F27613095C1068C2F2000340F272
:100C0000FA19B3F90030C2F20009A0EB203089F8DC
:100C10000010184440F2781301391060020BC2F240
:100C2000000305291A801BD840F30F30DFE801F0DC
:100C3000031C2022252907464042002624E0B1FB60
:100C4000F0F202FB101000287FF450AF40F27E104B
:100C5000C2F200000178B1FA81F14A09027040E75E
:100C60000026002700200FE04642074600200BE048
:100C7000464208E04742002606E04742064600207A
:100C800002E00646404200274FF6A534CFF6FF7437
:100C90002146A042C8BF014640F25B4501F26542D1
:100CA000A84240464FF00201C8BF4FF40C6202F068
:100CB000A3FB2046A742C8BF384600F26542404623
:100CC0000121AF42C8BF4FF40C6202F095FBA6426F
:100CD000C8BF344604F2654240460021AE42C8BF58
:100CE0004FF40C6202F088FB40F2F014C2F20004F0
:100CF000267899F800504AF6AB21701BC2F6AA215B
:100D000080FB012303EBD37202EB4202A0EB420013
:100D1000063080FB011202EBD27202EB420240F27B
:100D2000DC11A0EB420045F25A5240F20827C2F211
:100D30000001C0F60002C2F200070B6832F9102071
:100D400038689A1A43097C2B0A609CBF01303860CE
:100D50003868012E16D0012D14D104F041FA014655
:100D60004FF6EC10C4F2F84004F010F940F2002104
:100D7000022E08BF80F00040C2F20001086000208F
:100D8000386008E0B0F57A6F05D340F20020C2F277
:100D9000000000210160257001B0BDE8F08F000067
:100DA0004FF4407001F0CEBB80B540F61D1001F04D
:100DB000CDFD002818BF01F0D7FD40F6FF700221DD
:100DC00001F0B8FA012809D140F6FF7001F098FA55
:100DD000012803D101F08CFA012080BD002080BDE4
:100DE000B0B54FF4E16001F07DFC42F20004C4F2C2
:100DF0000004204601F0D6FF40F21C25C2F2000597
:100E000000204FF4001148F6A042C5E900102873F5
:100E10002046AA6002F0ACF82046294602F02CF8E1
:100E200013200021002201F097FB2046012102F04F
:100E300009F92046BDE8B04002F088B870B540F22C
:100E4000115001F04FFC40F2125001F04BFC40F207
:100E5000135001F047FC40F2165001F043FC4FF0F4
:100E60009040012100224FF4004301F0BDFA4FF001
:100E70009040002101224FF4004301F0DFFA40F2DC
:100E80000044C4F60004204601210022082301F09A
:100E9000ABFA204600210122082301F0CFFA4FF0DF
:100EA0009040012100224FF4805301F09DFA4FF051
:100EB0009040002101224FF4805301F0BFFA4FF01F
:100EC000904001210022022301F08EFA4FF0904061
:100ED00000210122022301F0B1FA4FF090400121DC
:100EE0000022012301F080FA4FF0904000210122FE
:100EF000012301F0A3FA04F58065284601210022B0
:100F00004FF4005301F070FA2846002101224FF4FB
:100F1000005301F093FA2046002100224FF40063B1
:100F200001F062FA2046002101224FF4006301F033
:100F300085FA04F58056304600210022022301F094
:100F400053FA304600210122022301F077FA2846A5
:100F5000002100224FF4804301F046FA2846002188
:100F600001224FF4804301F069FA4FF090400321D1
:100F70000022102301F038FA4FF0904000210122A6
:100F8000102301F05BFA4FF0904003210022402330
:100F900001F02AFA4FF0904000210122402301F095
:100FA0004DFA2046022100224FF4805301F01CFA32
:100FB0002046002103224FF4805301F03FFA2046DF
:100FC00002214FF4805201F07DFA4FF0904002214F
:100FD00000224FF4806301F007FA4FF090400021A7
:100FE00000224FF4806301F029FA4FF09040022173
:100FF0004FF4806201F066FA2046022100224FF48D
:10100000004301F0F1F92046002100224FF4004393
:1010100001F014FA204602214FF4004201F052FA86
:101020004FF09040022100224FF4007301F0DCF9F0
:101030004FF09040002100224FF4007301F0FEF9C0
:101040004FF0904002214FF4007201F03BFA20462D
:10105000022100224FF4804301F0C6F9204600210E
:1010600000224FF4804301F0E9F9204602214FF4B9
:10107000804201F027FA4FF09040022100224FF405
:10108000807301F0B1F94FF09040002100224FF43D
:10109000807301F0D3F94FF0904002214FF4807239
:1010A00001F010FA2046022100224FF4005301F013
:1010B0009BF92046002100224FF4005301F0BEF9B5
:1010C000204602214FF4005201F0FCF92046012194
:1010D0000022042301F088F9204600210122042384
:1010E00001F0ACF92046012100224FF4806301F0A9
:1010F0007BF92046002103224FF48063BDE8704055
:1011000001F09CB970B540F20B6001F0EBFA42F6C9
:101110000044C4F20104204601F044FE40F254258C
:10112000C2F2000500264FF4001040F6CA01C5E9DE
:1011300000062046A9602E7301F01AFF20462946BA
:1011400001F09AFE20460221002202F079F92046A1
:101150000121002202F074F920460021002202F051
:101160006FF920460221002202F04CF920460121AD
:10117000002202F047F920460021002202F042F945
:1011800020460221702202F019F920460121702226
:1011900002F014F920460021702202F00FF92046D7
:1011A0000221002202F028F920460121002202F04B
:1011B00023F920460021002202F01EF940F24425C6
:1011C000C2F200054FF40020C5F806004FF0007091
:1011D000C5F80A00204602212A4601F0DBFF20461E
:1011E00001212A4601F0D6FF204600212A4601F0BF
:1011F000D1FF40F22C21C2F200014FF400603C22EA
:10120000C1E9000601F108004FF480434CC02046BC
:101210004E6101F06DFF204601F09EFE2046022146
:10122000012202F095F920460121012202F090F9F5
:1012300020460021012202F08BF9204602210422DF
:1012400002F0ACF920460121042202F0A7F9204661
:101250000021042202F0A2F90D200021002201F059
:101260007BF92046012101F0EDFE2046BDE87040EB
:1012700001F06CBEF0B581B040F2096001F032FAC5
:101280004FF4A06001F02EFA032001F0CFFA0920FC
:10129000012100220127002501F05EF9002000F065
:1012A00071FE40F28411C2F2000140F27010C2F2ED
:1012B000000001F10C0C4FF4806242F24C448CE8C7
:1012C00025004FF440500223C4F2010408620020BC
:1012D0004FF4807681E8D000C1E9065300F076FE35
:1012E000002000F0B1FE002000F0D2FE002002211C
:1012F00000F0C0FF0020022100F0FEFE002000F000
:10130000D3FE0120022100F03FFC00200421022234
:1013100000F064FC01200621022200F05FFC0020A6
:1013200000F024FC0120012100F0FCFC01204FF41E
:10133000602100F01BFD00F0A7FB00F0B9FB00F0FE
:1013400009FE00F057FB00F06DFB00F07FFB4FF44F
:101350008070012101B0BDE8F04000F0D5BB00BFB6
:10136000F0B581B005464FF09040022101220423E0
:10137000012601F039F84FF09040002103220423A8
:10138000002701F05BF84FF090400121042201F0AA
:1013900099F84FF0904002210122082301F024F82F
:1013A0004FF0904000210322082301F047F84FF04E
:1013B00090400121082201F085F840F2117001F0FF
:1013C00091F94FF4A06001F08DF944F20044C4F2A9
:1013D00000042046294602F0B1FB2046002102F01D
:1013E000DBFB2046002102F0E3FB2046002102F057
:1013F000EBFB2046002102F06FFC2046082102F0A2
:10140000FBFB2046042102F0FFFB204602F0E8FB34
:101410000B200221002201F09FF8042000F0B2FD11
:1014200040F2A81140F26520C2F20001C2F20000B1
:10143000C1E902604FF4405004F124020862042024
:10144000C1E90027C1E90477C1E9067600F0BEFDD5
:10145000042000F0F9FD042000F01AFE204640218F
:1014600002F0E6FD0420022100F004FF0420012127
:1014700000F042FE042001B0BDE8F04000F014BED0
:1014800070B540F20044C4F600040546204602212F
:1014900000224023002600F0A7FF2046002103225F
:1014A000402300F0CBFF20460021402201F00AF843
:1014B000204602210022802300F096FF20460021D2
:1014C0000322802300F0BAFF20460021802200F092
:1014D000F9FF40F20E6001F005F94FF4A06001F051
:1014E00001F943F60004C4F201042046294602F043
:1014F00025FB2046002102F04FFB2046002102F090
:1015000057FB2046002102F05FFB2046002102F03D
:10151000E3FB2046082102F06FFB2046042102F085
:1015200073FB204602F05CFB0A200221002201F03E
:1015300013F8022000F026FD40F2A81140F26420CA
:10154000C2F20001C2F200000122C1E902204FF400
:10155000405004F1240308620220C1E90036C1E9C9
:101560000466C1E9066200F031FD022000F06CFD66
:10157000022000F08DFD2046402102F059FD02209E
:10158000022100F077FE0220012100F0B5FD0220CB
:10159000BDE8704000F088BD40F2F410C2F20000D7
:1015A000016801310160704740F21820C2F200006A
:1015B00000210160704700BF10B540F21820C2F250
:1015C00000000168B1F5FA6F0BD940F21424C2F2A1
:1015D0000004207810B90020FFF7B8F9012020702E
:1015E00007E040F21422C2F200020023013113701E
:1015F000016042F20000C4F200000121BDE8104089
:1016000001F036BD80B5012000F0C6FB42F6004077
:10161000C4F201000121BDE8804001F029BD00BFF6
:1016200080B5FFF7CFF90020022100F0DFFD002890
:1016300008BF80BD00200221BDE8804000F010BE40
:1016400080B50220022100F0D1FD002808BF80BD36
:1016500000F09EF802200221BDE8804000F000BEAC
:1016600080B50420022100F0C1FD002808BF80BD24
:1016700004200221BDE8804000F0F2BD40F2F410E9
:10168000C2F2000000687047002808BF704740F2AF
:10169000F411C2F200010A6800BF0B689B1A834272
:1016A000FAD37047704700BFFEE700BFFEE700BFF8
:1016B000FEE700BFFEE700BF704700BF704700BFF6
:1016C0007047000080B5FFF7D9FF40F2E411C2F285
:1016D00000010968401AB0F5FA7F98BF80BD40F25A
:1016E0000C20C2F200000021016040F20420C2F28E
:1016F0000000016080BD00BF10B584B04AF6CD3057
:10170000ADF8000040F20400C2F200000024002105
:101710000068C4F2C8248DF80210214603F0DCFDF5
:1017200003F02AFD40F28011C2F200010968ADF811
:1017300005000846214603F0CFFD03F01DFD40F2F1
:101740000021C2F200010968ADF8070008462146F1
:1017500003F0C2FD03F010FD40F2D811C2F2000107
:101760000A68ADF80300501C6C46086020460D2145
:10177000CDF8092000F008F9ADF80D0043F600009F
:10178000C4F2010021460F2200F0E6F804B010BDBB
:10179000B0B584B040F2E01040F26421C2F2000023
:1017A000C2F20001B0F900200978B2F1FF3F04DC79
:1017B0002F2940F0CE8000220280038840F270057D
:1017C0005A1C1CB2C2F20005002B0280295500F001
:1017D000C08091B2022912D1687840F2E311C2F2BE
:1017E00000010228087046D001283ED0002840F0B1
:1017F000B08040F2E210C2F20000082140E040F266
:10180000E211C2F20001097812B28A42C0F2A1804C
:101810002A4432F8024C4FF6FF7202800239284601
:1018200000F0B2F8844240F09480A878002840F09C
:101830009080FFF723FF40F2E311C2F20001097824
:1018400040F2E412C2F20002012910601BD0B1BBC9
:10185000B5F9030040F20421C2F20001086040F231
:101860000E01681DC2F2000127E040F2E210C2F250
:1018700000000B2104E040F2E210C2F200000A2155
:10188000017004B0B0BD40F20420B5F90310C2F2FB
:101890000000B5F90520016040F20C20C2F2000002
:1018A0000260E87940F20E01C2F20001087040F2D5
:1018B0000F0105F10800C2F20001007808704AF635
:1018C000CD30ADF8000040F20400C2F20000002468
:1018D00000210068C4F2C8248DF80210214603F0EC
:1018E000FBFC03F049FC40F28011C2F200010968E0
:1018F000ADF805000846214603F0EEFC03F03CFC81
:1019000040F20021C2F200010968ADF80700084664
:10191000214603F0E1FC03F02FFC40F2D811C2F2A3
:1019200000010A68ADF80300501C6C4608602046B0
:101930000D21CDF8092000F027F8ADF80D0043F691
:101940000000C4F2010021460F2200F005F8FFF765
:101950002BFE04B0B0BD0000F0B581B092B11446CA
:101960000D460646002700BFE95D304602F054F9F7
:10197000304640F2067102F099FB0028F8D001379A
:10198000A742F1D101B0F0BDB0B50022012917DBAB
:1019900041F2210E03788C46013982EA03220823A2
:1019A00014B25500002CA3F1010348BF8EEA420592
:1019B0001A062A46F4D1BCF1020F00F10100E9DA5F
:1019C00090B2B0BD40F27411C2F2000108707047CD
:1019D00040F27410C2F200000078704780B540F207
:1019E000093000F0BFFE40F20930BDE8804000F051
:1019F000C9BE00BF42F20840C4F201000168C90735
:101A000018BF7047016841F001010160704700BFD5
:101A100042F20840C4F20100016821F001010160B6
:101A2000704700BF42F20840C4F20100016841F073
:101A30000801016001680907FCD4016841F0040154
:101A4000016000BF01684907FCD4704742F20840BA
:101A5000C4F20100016841F480710160704700BF69
:101A600042F20840C4F20100016821F48071016073
:101A7000704700BF42F20840C4F20100016841F41F
:101A800000010160704700BF42F20840C4F201004B
:101A9000016821F400010160704700BF42F2084074
:101AA000C4F20100016841F080710160704700BF1D
:101AB00042F20840C4F20100016821F08071016027
:101AC000704700BF42F20442C4F2010213680228C8
:101AD00023F4C053136011D0012818BF7047106859
:101AE00020F4604010604FF4604000EB413011681A
:101AF00080B2084310604FF4006001E04FF4805062
:101B0000116808431060704742F20442C4F20102B7
:101B1000002900F4807105D0B9B941051BD48007B4
:101B20001FD4704719B1116821F48071116041050B
:101B300003D5116821F480611160800758BF704798
:101B4000506820F0020050607047116841F48071C5
:101B500011604105E3D5116841F48061116080078F
:101B6000DFD5506840F002005060704742F20841F3
:101B7000C4F201010A68002822F4006218BF02F5CD
:101B800000620A60704700BF022814D0012818BF05
:101B9000704742F22C40C4F20100026822F4700245
:101BA00002604FF4700202EB0151026801F470010F
:101BB00011430160704742F22C40C4F20100C26838
:101BC00022F44012C2604FF4401202EB0151C2688D
:101BD00001F440111143C160704700BF80B5B1F1FD
:101BE000120342F20C4C18BF0B460528C4F2010C3C
:101BF0000DD8DCF828E000EB80001F2181402EEAA0
:101C0000010103FA00F00843CCF8280020E00B287B
:101C10000ED800EB8000DCF824E01E381F21814044
:101C20002EEA010103FA00F00843CCF824000FE08B
:101C30000F280DD800EB8000DCF820E03C381F2195
:101C400081402EEA010103FA00F00843CCF820009D
:101C5000092B0CD8DCF8040003EB430107238B406D
:101C6000984302FA01F10843CCF8040080BD112B1F
:101C700088BF80BD03EB4301DCF800001E39072359
:101C80008B40984302FA01F10843CCF8000080BD74
:101C900080B542F2384CC4F2010CDCF80030DCF8BC
:101CA00000E0C3F30153181A00EB8000C0F10F00ED
:101CB0001F2383402EEA030301FA00F01843092989
:101CC000CCF800000CD85CF8280C01EB410107238C
:101CD0008B40984302FA01F108434CF8280C80BD70
:101CE000122988BF80BD01EB41015CF82C0C1E3924
:101CF00007238B40984302FA01F108434CF82C0C5F
:101D000080BD00BF42F21442C4F20102536AC3F321
:101D10000153C01A033003289CBF6FF31F3142F8F0
:101D20002010704742F20842C4F20102002900F07C
:101D3000010103D079B9800713D4704719B1116834
:101D400021F480111160800758BF7047106820F49B
:101D5000004010607047116841F4801111608007E5
:101D6000EBD5106840F4004010607047012805D0A2
:101D7000022818BF70476FF4E04001E06FF4602064
:101D800042F20842C4F20102136818401060106861
:101D900008431060704700BFC10742F20841C4F217
:101DA000010103D00A6842F480020A60800758BF2C
:101DB0007047086840F400100860704742F24C40D9
:101DC000C4F20100006880B2704700BF03280AD83F
:101DD000DFE800F0020C131A42F23C40C4F20100AA
:101DE000006880B27047002080B2704742F23C40E9
:101DF000C4F20100406880B2704742F23C40C4F235
:101E00000100806880B2704742F23C40C4F2010099
:101E1000C06880B2704700BF42F20041C4F20101C5
:101E20000968084018BF0120704700BF42F2004116
:101E3000C4F201010A6822EA00000860704700BF8E
:101E4000012807D0042807D002281CBF00207047B3
:101E5000202102E0402100E0802142F20042C4F251
:101E60000102136852681840114018BF0121002870
:101E700018BF01200840704742F20041C4F201013E
:101E80000A6822EA00000860704700BFC10742F2FA
:101E90000441C4F2010103D00A6842F040020A6022
:101EA000820703D50A6842F020020A60400758BF43
:101EB0007047086840F0800008607047C10742F230
:101EC0000441C4F2010103D00A6822F040020A6012
:101ED000820703D50A6822F020020A60400758BF33
:101EE0007047086820F080000860704742F20441A3
:101EF000C4F201010A684FF6E053CFF63F731A406F
:101F00000A600A6810430860086840F4400040F422
:101F100000700860704700BF42F20441C4F2010142
:101F20000A684FF6FF53CFF63F7301381A40C3B229
:101F3000022B0A6088BF704740B203A252F820000B
:101F40000A681043086070470000800000004000ED
:101F50000000C00042F20440C4F2010001684FF6E4
:101F6000E052CFF63F7211400160704742F22442C6
:101F70006FF31F30C4F201026FF31F315060116024
:101F800070470000042200EB8001C4F2020202EB61
:101F900081014B68800023F001034B6000234B60FC
:101FA0008B60CB600B610F21136801FA00F01843BE
:101FB0001060704700210122C0E90011C0E9022130
:101FC000C0E90412C0E906110162704710B540F281
:101FD000080ED1F800C000EB8000C4F2020E0EEB38
:101FE0008003C3F808C0CA68DA60CA695A605EF83C
:101FF00020204B6822F47C5C0A690C6A43EA0C03DB
:102000001A4322434EF820208A685EF82030002AC6
:1020100023F0400308BF40334EF820304A695EF891
:102020002030002A23F0800308BF80334EF8203090
:1020300089695EF82020002922F0100218BF1032B2
:102040004EF8202010BD00BF082100EB8000C4F234
:10205000020151F8202042F0200241F82020704770
:10206000082100EB8000C4F2020151F8202022F088
:10207000200241F820207047082100EB8000C4F2C4
:10208000020151F8202042F4804241F8202070479C
:10209000082100EB8000C4F2020151F8202022F454
:1020A000804241F820207047082100EB8000C4F2F4
:1020B000020151F8202042F0010241F8202070472F
:1020C000082100EB8000C4F2020151F8202022F028
:1020D000010241F820207047102200EB8000C4F27A
:1020E000020242F820107047142200EB8000C4F274
:1020F000020242F8201070470C2200EB8000C4F26C
:10210000020242F8201070470C2100EB8000C4F25C
:10211000020151F820007047082200EB8000C4F251
:10212000020252F8203023F44053194342F82010A1
:10213000704700BF082200EB8000C4F2020252F890
:10214000203023F44063194342F82010704700BF49
:10215000082200EB8000C4F2020252F8203023F47F
:102160004073194342F82010704700BF082100EB6C
:102170008000C4F2020151F8202042F0800241F8B0
:1021800020207047082100EB8000C4F2020151F8C2
:10219000202022F0800241F820207047082100EB27
:1021A0008000C4F2020151F8202042F0400241F8C0
:1021B00020207047082100EB8000C4F2020151F892
:1021C000202022F0400241F820207047082200EB36
:1021D0008000C4F2020252F82030002923F01003DC
:1021E00018BF103342F82030704700BF80B54B1E37
:1021F000072B4FF0000131D840F2000CC4F2020C62
:10220000DFE803F0040E2C132C2C2C18DCF8001043
:1022100082000F239340194021FA02F30E2113E0AC
:10222000DCF800E08300022108E0DCF800E0830035
:10223000042103E0DCF800E08300082101FA03F246
:1022400002EA0E0222FA03F300EB80000CEB80009E
:102250008068084010EA030118BF0121084680BDCC
:102260000422C4F202028000136801FA00F018434D
:1022700010607047082200EB8000C4F2020252F89E
:102280002030194342F82010704700BF082200EBAD
:102290008000C4F2020252F8203023EA010142F821
:1022A000201070470022C4F202021268800001FA76
:1022B00000F0104018BF0120704700BF0422C4F294
:1022C00002028000136801FA00F0184310607047A2
:1022D00043F20000C4F2000000210160704700BF1B
:1022E00043F20000C4F200004AF6AA2101607047E0
:1022F00043F20000C4F200004CF6CC41016070478C
:1023000043F20001C4F2000145F255520A60022274
:10231000CFF6F072CB6803F004031AB1002B02F180
:102320000102F7D1002B11BF00206FF31F300861AD
:102330000120704780B540F2020ECFF6F07E43F2E6
:10234000000CC4F2000C45F255527346CCF8002044
:10235000DCF80C2002F001021BB1002A03F101039A
:10236000F6D16AB9CCF80410DCF80C10BEF1000FFD
:1023700001F0020103D000290EF1010EF4D109B1E0
:10238000002080BD6FF31F30CCF808004AF6AA2069
:10239000CCF80000012080BD43F20C01C4F2000122
:1023A0000968084018BF01207047000000F138405C
:1023B0004FEAB020052888BF7047C1B22F2222FA09
:1023C00001F1C90700D1704710B545F26651C0F65A
:1023D000000131F81040204600F0C4F92046BDE865
:1023E000104000F0CFB900BF2DE9F041D0F800E077
:1023F000D0F80CC000244FF00308002605E000BF11
:102400000136102E04F1020412D023FA06F7FF075A
:10241000F6D008FA04F72EEA070E01FA04F54EEAA0
:10242000050E2CEA070702FA04F547EA050CE7E770
:10243000C0F800E0C0F80CC0BDE8F081B0B50129DB
:10244000416814BF994319434160D0F808C0002186
:102450004FF0030E002404E00134102C01F10201BE
:102460000CD023FA04F5ED07F6D00EFA01F52CEAAC
:10247000050C02FA01F54CEA050CEDE7C0F808C0BE
:10248000B0BD00BF81617047816270471823002A88
:1024900008BF282319507047416170470069084000
:1024A00018BF0120704700BF006980B2704700BFAD
:1024B0004069084018BF0120704700BF406980B2E2
:1024C000704700BFF0B5D0F820E0D0F824C000235A
:1024D0000F27002505E000BF0135082D03F1040397
:1024E0000CD022FA05F6F607F6D007FA03F62EEA24
:1024F000060601FA03F446EA040EEDE70823002479
:102500000F2504E00133102B04F104040CD022FA4F
:1025100003F6F607F6D005FA04F62CEA060701FAE8
:1025200004F647EA060CEDE7C0F820E0C0F824C046
:10253000F0BD00BF41F48032C261C161C261C169B6
:10254000C069704740F080604EF60C5140F0FD705D
:10255000CEF20001086070474EF60C5CCEF2000C23
:10256000DCF8003003F4E063B3F5E06F03D14FF023
:10257000000C04232BE0DCF8003003F4E063B3F537
:10258000C06F03D14FF0010C032320E0DCF80030D2
:1025900003F4E063B3F5A06F03D102234FF0020C04
:1025A00015E0DCF8003003F4E063B3F5806F03D18D
:1025B0004FF0030C01230AE0DCF800304FF0040C6C
:1025C00003F4E063B3F5407318BF01239B00994007
:1025D0000F2323FA0CF31A4011434EF20012CEF2ED
:1025E0000002090140EA020383F8001300F01F0112
:1025F000012303FA01F11C2303EAD0008150704744
:1026000000F01F01012202FA01F14EF28012CEF217
:10261000000242EAD00020F003000160704700BFD2
:102620004FF68072C1F6FF72114008434EF6085112
:10263000CEF20001086070474EF61051CEF2000154
:102640000A681043086070474EF61051CEF2000140
:102650000A6822EA00000860704700BF4EF21001CD
:10266000CEF200010A68042822F0040208BF0432F6
:102670000A60704741F20400C4F2020050F8041CE2
:1026800041F0010140F8041C50F8041C8907FBD5F7
:1026900001680C22C0F6FF021140016001684FF68C
:1026A000FF72CFF2C0721140016001684FF6FF72F5
:1026B00021F44001016050F8041CCFF6F262114091
:1026C00040F8041C816A40F2431221F00F0181623C
:1026D000C16A9143C162016B21F0010101630021D4
:1026E0004160704741F2000300F01F018009C4F20D
:1026F00002034FF0010CC2580CFA01F11143C15012
:10270000704700BF41F2000300F01F018009C4F2CE
:1027100002034FF0010CC2580CFA01F122EA010148
:10272000C150704741F2000300F01F018009C4F25C
:1027300002034FF0010CC2580CFA01F11143C150D1
:10274000704700BF41F2000300F01F018009C4F28E
:1027500002034FF0010CC2580CFA01F122EA010108
:10276000C150704741F2000300F01F018009C4F21C
:1027700002034FF0010CC2580CFA01F11143C15091
:10278000704700BF41F2000300F01F018009C4F24E
:1027900002034FF0010CC2580CFA01F122EA0101C8
:1027A000C150704741F22000C4F20200016841F4B8
:1027B00080310160704700BF41F22000C4F2020086
:1027C000016821F480310160704700BF41F20401CB
:1027D000C4F202010A6822F0030210430860704745
:1027E00041F20400C4F20200006800F00C007047DF
:1027F00041F20401C4F202010A6822F0F00210431F
:102800000860704741F20401C4F202010A6822F430
:10281000E06210430860704741F20401C4F2020113
:102820000A6822F4605210430860704741F20401C4
:10283000C4F202010A68042822F440420A60CA6A0B
:1028400022F48072CA6288BF7047DFE800F0030894
:102850000A0E1200C86A20F48070C86270470868C7
:102860000AE0086840F4804006E0086840F4004050
:1028700002E0086840F440400860C86A40F4807094
:10288000C862704741F20401C4F202010A6822F4EE
:1028900040020A600A6810430860704741F204026F
:1028A000C4F202021368084323F077431843106010
:1028B000704700BF41F20402C4F20202D2F800C025
:1028C0004FF6FF73CFF2C27303EA0C031360136871
:1028D000084318431060704741F23001C4F202010E
:1028E0000A6822F003020A600A6810430860704711
:1028F00041F23001C4F202010A6822F040020A608B
:102900000A6810430860704741F22001C4F20201D6
:102910000A6822F440720A600A681043086070472F
:1029200041F22C01C4F202010A6822F00F021043A6
:102930000860704741F22001C4F202010A6822F0E7
:1029400018020A600A6810430860704741F20002EA
:102950008109C4F20202895800F01F0021FA00F038
:1029600000F00100704700BF41F22400C4F20200F1
:10297000016841F080710160704700BF41F20801B9
:10298000C4F202010968084018BF0120704700BF67
:1029900041F20801C4F202010A681043086070475E
:1029A00041F20801C4F202010A681043086070474E
:1029B00041F20801C4F202010A6822EA000008603C
:1029C000704700BF0146B0F5006F4FF000001DDA00
:1029D000E1B3102950D0182940F0958041F2000C45
:1029E0004FF6FE71C4F2020CC0F20F01002200BFCC
:1029F000DCF80000013942F10003800101D4002B12
:102A0000F6D1DCF80000C0F3406070474AD0B1F561
:102A1000106F61D0B1F5506F18BF704741F2000CD4
:102A20004FF6FE71C4F2020CC0F20F01002200BF8B
:102A3000DCF83400013942F10003800701D4002B97
:102A4000F6D1DCF83400C0F34000704741F2000CCE
:102A500040F2FF40C4F2020C002200BFDCF800107C
:102A6000013842F10003890701D4002BF6D1DCF8CC
:102A70000000C0F34000704741F2000C40F2FF70CC
:102A8000C4F2020C002200BFDCF80010013842F151
:102A90000003890301D4002BF6D1DCF80000C0F359
:102AA000404070474FF6FE7141F2000CC0F20F013A
:102AB000C4F2020C01F17C71002200BFDCF820009E
:102AC000013942F10003800701D4002BF6D1DCF874
:102AD0002000C0F34000704741F2000C4FF6FE7139
:102AE000C4F2020CC0F20F01002200BFDCF8240087
:102AF000013942F10003800701D4002BF6D1DCF844
:102B00002400C0F34000704741F2000300F01F01B1
:102B10008009C4F202034FF0010CC2580CFA01F113
:102B20001143C150704700BF41F2000300F01F0184
:102B30008009C4F202034FF0010CC2580CFA01F1F3
:102B400022EA0101C1507047B0F5006F0FD0102884
:102B500018BF704741F20000C4F202000168026829
:102B600041F4802122F4803202600160704741F21A
:102B70000000C4F20200016A026A41F0040122F07E
:102B80000102026201627047B0F5006F0FD0102899
:102B900018BF704741F20000C4F2020001680268E9
:102BA00021F4802122F4803202600160704741F2FA
:102BB0000000C4F20200016A026A21F0040122F05E
:102BC000010202620162704741F20000C4F2020099
:102BD000016841F400210160704700BF41F200002C
:102BE000C4F20200016821F400210160704700BFB7
:102BF00041F20001C4F202010A6822F0F80242EA3E
:102C0000C0000860704700BF41F23401C4F2020105
:102C10000A6822F0F80242EAC0000860704700BF6C
:102C200041F20010C4F20200016800210160016855
:102C300043F64D42C1F62B2211430160704700BF9D
:102C400041F23411C4F202010A6822F007020A605C
:102C50000A6810430860704741F23811C4F202015B
:102C60000A6822F001020A600A681043086070478F
:102C700070B541F20402C4F202020146106841F24A
:102C8000002CC0F27A0C00F00C000828634619D121
:102C90001068136815681B014FF01103C0F38340DF
:102CA00058BF0223ED03184405D440F60013C0F2C8
:102CB0003D03434306E0936A03F00F030133BCFB7B
:102CC000F3F343431468D2F800E0106806291ED8D5
:102CD000C4F303142FA52C5D45F27255C0F6000510
:102CE000C0F3C220285C23FA04F424FA00F0DFE8E1
:102CF00001F00410123A06182000184670BDD16A7F
:102D0000C90531D449F68070C0F2D50070BD0020ED
:102D100070BD204670BDCEF30220285C24FA00F07E
:102D200070BDD06A40064FF4004058BF48F2120010
:102D300070BDD16A890708BF70BDD06A00F003007A
:102D4000012818460FD0D06A00F00300022804BF03
:102D50004FF4004070BDD06A00F00300032818BF94
:102D60004FF0000C604670BD1168C1F38131DFE89F
:102D700001F00204060E400870BD800870BD4AF6DE
:102D8000AB21CAF6AA21A0FB0101880870BDC008CA
:102D900070BD00BF0000000000000000010203043D
:102DA0000607080910B542F6FF31C4F20101884256
:102DB00011DC40F6FF71C4F20001884220DCB0F162
:102DC000804F3CD040F20041C4F20001884249D11A
:102DD00040F201443EE044F2FF31C4F20101884276
:102DE0001DDC42F60041C4F2010188422AD044F2BF
:102DF0000001C4F20101884234D14FF4447429E047
:102E000041F20001C4F2000188421ED042F20001EA
:102E1000C4F20001884225D14FF481641AE044F2E3
:102E20000041C4F20101884212D044F60001C4F20C
:102E30000101884218BF10BD40F212340AE04FF47D
:102E4000806407E040F20B3404E040F2044401E007
:102E500040F211342046FFF785FC2046BDE81040C3
:102E6000FFF790BC10BD00BF00214FF6FF72C0E914
:102E700000118260017370470A8842F6004CB0F17D
:102E8000804FC4F2010C826218BF60452ED10368E6
:102E900023F0700303604B8802681A4302608A883B
:102EA00003681A43026042F6FF338A68C4F20103E2
:102EB0009842C2620ADD44F2FF32C4F2010290423B
:102EC0001BDC604525D044F200021EE0B0F1804FCB
:102ED0001FD040F20042C4F20002904219D042F2E8
:102EE0000002C4F20002904213D02AE040F20043F4
:102EF000C4F200039842CAD0D5E744F60002C4F2F7
:102F00000102904205D044F20042C4F20102904214
:102F100017D1026822F440720260CA880368134322
:102F2000A0F18042A2F596324FEAB222072A03604E
:102F300007D8012303FA02F212F0E10F1CBF097B4C
:102F40000163416941F0010141617047016841F04D
:102F500001010160704700BF016821F001010160BB
:102F6000704700BF016841F080010160704700BFF9
:102F7000016821F080010160704700BF016821F005
:102F800002010160704700BF016841F00201016069
:102F9000704700BF026822F06002026002681143BD
:102FA00001607047016821F010010160704700BFA7
:102FB000016841F010010160704700BF002A816282
:102FC00018BF7047416941F001014161704700BF7E
:102FD00001637047C162704741627047406A704741
:102FE000806A80B2704700BF012907D0002918BF4E
:102FF0007047016841F0080101607047016821F0E5
:1030000008010160704700BF012907D0002918BFDF
:103010007047016841F0040101607047016821F0C8
:1030200004010160704700BF39B1012918BF704722
:10303000816841F0080181607047816821F00801D2
:1030400081607047C2681143C1607047C26822EA5C
:103050000101C160704700BFC26800690A400840B2
:1030600018BF0120002A18BF01221040704700BF7E
:10307000C9430161704700BF0069084018BF0120C3
:10308000704700BFC9430161704700BFC268114368
:10309000C1607047C26822EA0101C160704700BF89
:1030A000012907D0002918BF7047416841F0080185
:1030B00041607047416821F008014160704700BFDE
:1030C000D0F848C041F61F732CEA03038364836C75
:1030D000114319438164704742691143416170474C
:1030E0000021C0E90011C0E90211C0E904117047D4
:1030F00010B5D1E900230C891A434B89D1E903CEDD
:1031000022431A43496942EA0C0242EA0E02114381
:10311000416410BD416C41F480514164704700BF6F
:10312000416C21F480514164704700BF416C41F40F
:1031300080414164704700BF416C21F4804141648B
:10314000704700BF426C012922F4004208BF02F51B
:1031500000424264704700BF4268012922F0010228
:1031600008BF013242607047012907D0002918BF0B
:103170007047416821F0040141607047416841F0A7
:1031800004014160704700BF00218181C0E9001146
:1031900081607047032900F20F81DFE801F0028DA2
:1031A00046D4016A21F001010162816921F0030125
:1031B00081611168036A19430162016A21F0020109
:1031C0000162D188036A0B43A0F18041A1F59631D9
:1031D0004FEAB1210729036200F2EE80012303FACE
:1031E00001F111F0E10F00F0E780016A21F0040124
:1031F00001629188036A19430162016A21F00801A2
:1032000001621189036A1943016250F8041F21F415
:10321000807101605189036819430160016821F4DC
:103220000071016093890268C3E0016A42F6044CB0
:1032300021F480710162C169C4F2010C21F0030123
:10324000C1611168036A43EA01210162016A21F444
:1032500000710162D388016A41EA0321ACF10403E1
:103260009842016240F0A880016A21F48061016205
:103270009188036A43EA01210162016A21F4006135
:1032800001621189036A43EA01210162DCF800004E
:1032900020F48050CCF800005089DCF8001041EA9E
:1032A0000010CCF80000DCF8000020F40050CCF84E
:1032B0000000908902016DE0016A21F010010162B5
:1032C000816921F4407181611168036A43EA011147
:1032D0000162016A21F020010162D188036A43EA98
:1032E000011144F20003C4F201039842016255D077
:1032F00042F60041C4F2010188425DD1016A21F029
:10330000400101629188036A43EA01110162016A86
:1033100021F0800101621189036A43EA011101620F
:1033200042F60440C4F20100016821F480610160AA
:103330005189036843EA81010160016821F4006159
:103340000160918933E0016A42F6044C21F4805116
:103350000162C169C4F2010C21F44071C1611168BC
:10336000036A43EA01310162016A21F400510162FA
:10337000D388016A41EA0331ACF104039842016247
:1033800018BF7047DCF8000020F48040CCF8000043
:1033900050898201DCF8003060460AE044F2040003
:1033A000C4F20100016821F4806101605189036861
:1033B0008A0042EA03010160704700BF032988BF09
:1033C0007047DFE801F0020E050B50F8181F01E00E
:1033D00050F81C1F21F07001016008E050F81C1F1C
:1033E00001E050F8181F21F4E04112020160016869
:1033F00011430160704700BF03299CBF00EB8100AF
:1034000042637047032988BF7047DFE801F0020E6E
:10341000050B50F8181F01E050F81C1F21F008019F
:10342000016008E050F81C1F01E050F8181F21F45B
:10343000006112020160016811430160704700BF22
:10344000032988BF7047DFE801F0020E050B50F832
:10345000181F01E050F81C1F21F00401016008E072
:1034600050F81C1F01E050F8181F21F4806112026F
:103470000160016811430160704700BF032988BFE4
:103480007047DFE801F0020E050B50F8181F01E04D
:1034900050F81C1F21F08001016008E050F81C1F4B
:1034A00001E050F8181F21F4004112020160016888
:1034B00011430160704700BF032988BF7047DFE8F0
:1034C00001F00216080F50F8201F21F002010160E0
:1034D00013E050F8201F120221F4007101600CE08B
:1034E00050F8201F120321F40051016005E050F84C
:1034F000201F120121F020010160016811430160C9
:10350000704700BF032988BF7047DFE801F002164B
:10351000080F50F8201F21F00801016013E050F857
:10352000201F120221F4006101600CE050F8201FFE
:10353000120321F40041016005E050F8201F120140
:1035400021F080010160016811430160704700BFF4
:10355000032988BF7047DFE801F00216080F50F812
:10356000201F21F00101016013E050F8201F12021A
:1035700021F4807101600CE050F8201F120321F447
:103580008051016005E050F8201F120121F0100168
:103590000160016811430160704700BF02290AD031
:1035A00001290FD0002918BF704750F8201F21F0C3
:1035B000040101600CE050F8201F120221F4806128
:1035C000016005E050F8201F120121F04001016068
:1035D00001681143016070474FF4803101600021A0
:1035E00041607047F0B5032900F28B80DFE801F0FD
:1035F000021B355784465CF8203F4FF0010E23F044
:103600000103CCF80030DCF8003023F00A03CCF8DA
:1036100000301388DCF800703B43CCF800300346E0
:1036200053F8187F32E084465CF8203F4FF0100ECC
:1036300023F01003CCF80030DCF8003023F0A003B6
:10364000CCF800301388DCF8007047EA0313CCF89C
:103650000030034653F8187F3AE084465CF8203F78
:103660004FF4807E23F48073CCF80030DCF8003017
:1036700023F42063CCF800301388DCF8007047EAAC
:103680000323CCF80030034653F81C7F27F00307D0
:103690001F6054881D6804266FF0F00721E08446FF
:1036A0005CF8203F4FF4805E23F48053CCF8003068
:1036B000DCF8003023F42043CCF800301388DCF829
:1036C000007047EA0333CCF80030034653F81C7F00
:1036D00027F440771F6057881C683D020C266FF462
:1036E00070472C431C601C683C401C60D4881D68DB
:1036F000B4402C431C60DCF8003043EA0E03CCF8E5
:103700000030032988BFF0BD9288DFE801F0020590
:10371000080E50F8181F04E050F8181F07E050F882
:103720001C1F21F00C01016005E050F81C1F21F462
:10373000406112020160016811430160F0BD00BFE9
:10374000032988BF7047DFE801F0020E050B50F82F
:10375000181F01E050F81C1F21F00C01016008E067
:1037600050F81C1F01E050F8181F21F440611202AC
:103770000160016811430160704700BF03298EBFDB
:10378000002000EB8100406B704700BF70B51488CB
:103790005688B4FA84F34FF0010E5B09012E08BF7E
:1037A0004FF0020E056A00294FEA430C4FD025F076
:1037B00010010162016A21F0A0010162016A41EA7F
:1037C00004110162014651F8183F23F440730B6065
:1037D0000B6843EA06230B600B6823F470430B600D
:1037E000D3880C6844EA03340C60046A44F0100483
:1037F000046292880C6824F440640C600C6844EA0B
:1038000002240C60046A24F001040462046A24F0B7
:103810000A040462046A44EA0C0606620E6826F092
:1038200003060E600E6846EA0E060E600E6826F06D
:10383000F0060E600E6846EA03130B60036A43F05D
:1038400001030362086820F00C0008604CE025F0DA
:1038500001010162016A21F00A010162016A21434A
:103860000162014651F8183F23F003030B600B6817
:1038700033430B600B6823F0F0030B60D3880C68B4
:1038800044EA03140C60046A44F001040462928860
:103890000C6824F00C040C600C6814430C60046A7F
:1038A000120224F010040462046A24F0A0040462EA
:1038B000046A44EA0C1606620E6826F440760E602E
:1038C0000E6846EA0E260E600E6826F470460E60FC
:1038D0000E6846EA03330B60036A43F01003036289
:1038E000086820F44060086008681043086070BDF4
:1038F000012907D0002918BF7047416841F08001B5
:1039000041607047416821F080014160704700BF0D
:10391000826822F070028260826811438160704781
:10392000426822F070024260426811434160704771
:10393000826822F0070282608268114381607047CA
:10394000012907D0002918BF7047816841F0800124
:1039500081607047816821F080018160704700BFFD
:10396000D0F808C011432CF43F4CC0F808C0D0F880
:1039700008C041EA0C018160816841EA032181604D
:10398000704700BFD0F808C042EA03122CF0070CC1
:10399000C0F808C0D0F808C041EA0C018160D0F836
:1039A00018C040F203312CEA01018161D0F818C03F
:1039B00040F2011141EA0C018161016A21F00A0122
:1039C0000162016A21F0A0010162016A11430162F2
:1039D000704700BF816821F007018160704700BF18
:1039E000826822F07002826082681143816081687F
:1039F00021F007018160816841F007018160704713
:103A0000F0B5066A602911D126F010060662066A32
:103A1000120126F0A006066210244FF00C0C6FF481
:103A2000704E4FF480756FF440760EE026F001067C
:103A30000662066A4FF0040C26F00A0606626FF072
:103A4000F00E01256FF003060124076A03FA0CF358
:103A50003A43026282693240826182692A4382610A
:103A6000826902EA0E02826182691A438261026AF5
:103A700022430262826822F07002826082681143EF
:103A80008160816821F007018160816841F0070150
:103A90008160F0BDD0F808C011432CF43F4CC0F851
:103AA00008C0D0F808C041EA0C018160816841EA91
:103AB00003218160816821F077018160816841F094
:103AC00077018160704700BFD0F808C011432CF423
:103AD0003F4CC0F808C0D0F808C041EA0C01816032
:103AE000816841EA03218160816841F480418160FD
:103AF000704700BF816821F480418160704700BF3A
:103B00000165704710B543F60001C4F20101884217
:103B100009D044F20041C4F20001884218BF10BD30
:103B200040F2114401E040F20E342046FEF71AFE46
:103B30002046BDE81040FEF725BE00BFB0B50446E4
:103B400043F60000C4F2010084420D4607D044F25F
:103B50000040C4F20000844205D1022000E00620AB
:103B6000FFF786F800E000202168090406D400EB86
:103B70005500B0FBF5F080B2E060B0BD400000EB56
:103B80005500B0FBF5F04FF6F0710140C0F3420074
:103B90000844E060B0BD00BF026822F0010202608C
:103BA000026822F4C062026002681143016070473B
:103BB000026822F001020260026822F48052026070
:103BC0000268114301607047026822F0010202603E
:103BD000426822F44052426042681143416070479B
:103BE000016841F001010160704700BF016821F0E8
:103BF00001010160704700BF026822F00802026004
:103C00000268114301607047026822F004020260FA
:103C100002681143016070476FF35F218162704752
:103C2000406A6FF35F207047026801F4002122F0C0
:103C300001020260426822F400224260426811439D
:103C4000416070470268072922F00102026088BFC4
:103C50007047DFE801F004090E13181D22274168A0
:103C600041F4802141607047416821F48021416026
:103C70007047416841F4003141607047416821F468
:103C8000003141607047416841F4803141607047C4
:103C9000416821F4803141607047416841F400413E
:103CA00041607047416821F400414160704700BFA6
:103CB000016821F001010160816821F48051816077
:103CC000704700BF016821F001010160816841F483
:103CD00080518160704700BF026822F001020260DB
:103CE000026822F4004202600268114301607047DA
:103CF000026822F001020260826822F4006282609F
:103D00008268114381607047416841F480114160CD
:103D1000704700BF416821F480114160704700BFC7
:103D2000426822F4C0024260426811434160704719
:103D3000016841F400510160704700BF016821F43F
:103D400000510160704700BF026822F0010202606A
:103D5000026822F400620260026811430160704749
:103D6000026801F0100122F001020260426822F0B4
:103D7000100242604268114341607047026822F0BD
:103D800001020260426822F07F424260426842EAD9
:103D900001614160704700BF416841F4000141602A
:103DA000704700BF416821F400014160704700BFC7
:103DB000426902F07F4242614269114341617047AA
:103DC000016821F001010160416841F480414160D6
:103DD000704700BF016821F001010160416821F4D2
:103DE00080414160704700BF026801F0200122F06D
:103DF000010202604268114341607047016821F08E
:103E000001010160816841F008018160704700BFD5
:103E1000016821F001010160816821F008018160E1
:103E2000704700BF016821F001010160416841F461
:103E300000614160704700BF016821F0010101602D
:103E4000416821F400614160704700BFD0F800C0B4
:103E500001F480712CF0010CC0F800C0D0F804C04F
:103E600002F400722CF4E06CC0F804C0D0F804C076
:103E700041EA0C014160416811434160416803F42B
:103E80008062114341607047016821F001010160C7
:103E9000816841F020018160704700BF016821F016
:103EA00001010160816821F020018160704700BF3D
:103EB000016821F001010160816841F01001816019
:103EC000704700BF016821F001010160816821F0A5
:103ED00010018160704700BF0268090222F00102F0
:103EE0000260026989B222F47F42026102691143D1
:103EF00001617047426922F07F424261426942EAB1
:103F000001614161704700BF026801F0070122F0C2
:103F100001020260826822F460228260826842EAC2
:103F200041418160704700BF016821F001010160DB
:103F3000816841F002018160704700BF016821F093
:103F400001010160816821F002018160704700BFBA
:103F5000026801F0040122F001020260826811434C
:103F600081607047026822F001020260026922F05B
:103F7000FF0202610269114301617047026822F089
:103F800001020260826822F48072826082681143BA
:103F900081607047026822F001020260826822F4A8
:103FA000007282608268114381607047016821F06D
:103FB00001010160816841F480418160704700BF68
:103FC000016821F001010160816821F48041816074
:103FD000704700BF026801F01F0122F00102026079
:103FE000026822F078720260026842EA4151016080
:103FF000704700BF026801F01F0122F00102026059
:10400000026822F4F8120260026842EA014101608B
:10401000704700BF026801F4004122F00102026013
:10402000826822F400428260826811438160704796
:10403000826822F04002826082681143816070478A
:10404000826822F08002826082681143816070473A
:10405000016821F001010160816841F40051816033
:10406000704700BF016821F001010160816821F4FF
:1040700000518160704700BF016841F0020101609A
:10408000704700BF016821F002010160704700BF66
:10409000026801F4401122F001020260826822F4F9
:1040A0004012826082681143816070478A0910580B
:1040B00001F01F01C84000F00100704701F01F012E
:1040C0000122036A02FA01F119430162704700BF3D
:1040D00001F01F02C1F389114FF0010C0B580CFACB
:1040E00002F21A430A50704701F01F02C1F389110E
:1040F0004FF0010C0B580CFA02F223EA02020A50AC
:10410000704700BF8269114381617047C1F3891212
:1041100052F800C08A0D105801F01F03C1F304418A
:10412000C8402CFA03F1084000F00100704700BFBE
:10413000C1F304410122036A02FA01F11943016249
:10414000704700000948804709480047FEE7FEE73E
:10415000FEE7FEE7FEE7FEE7FEE7FEE7FEE7FEE737
:1041600004480549054A064B704700008541000890
:104170006901000868020020680A00206806002023
:104180006806002041F20400C4F2020050F8041C4A
:1041900041F0010140F8041C50F8041C8907FBD5CC
:1041A00001680C22C0F6FF021140016002684FF660
:1041B000FF71CFF2C0710A40026002684FF6FF73D0
:1041C00022F44002026050F8042CCFF6F2631A4049
:1041D00040F8042C826A40F2431322F00F028262FC
:1041E000C26A01F500319A43C262026B22F00102F9
:1041F0000263002242600268026002680260026894
:104200000260026811400160016841F0006141F400
:104210008021016050F8041C41F0807140F8041CBA
:1042200050F8041C8901FBD5016821F003010160ED
:10423000016841F00201016001680907FCD570477F
:1042400041F20400C4F20200016801F00C010829E7
:1042500041F20021C0F27A011AD1D0F800C00368FF
:1042600002681B014FF0110358BF0223D203CCF3A5
:1042700083421A4405D440F60011C0F23D01514377
:1042800006E0836A03F00F030133B1FBF3F15143FE
:1042900040F20002C2F200021160006804A1C0F303
:1042A0000310085C116821FA00F01060704700BF2D
:1042B00000000000000000000102030406070809D6
:1042C000704770477047754600F02CF8AE46050001
:1042D0006946534620F00700854618B020B5FFF721
:1042E0003FFFBDE820404FF000064FF000074FF0C1
:1042F00000084FF0000BAC46ACE8C009ACE8C009C0
:10430000ACE8C009ACE8C00921F007018D46704750
:1043100010B50446AFF300802046BDE81040FBF71F
:104320006ABF0000004870471000002001491820B3
:10433000ABBEFEE7260002007047000021F00042FD
:1043400001F00043A2F16052B2F5801F28BFD2F104
:104350007F6C0BD95FEA001C43EAC20242EB50704B
:1043600018BF704728BF20F001007047B2F5801FCA
:10437000BCBF184670474FEA410C1CF5001F02D223
:10438000084601F070B870B500F0D0FB000000895D
:10439000FFF7F6BF4FF00040A0F580007047000027
:1043A00010B591EA030F48BF83F0004300F11A846F
:1043B000841A71EB030C05D2121943EB0C03001B9A
:1043C00061EB0C014FEA1154A4EB135CDFF81CE124
:1043D0001EEA430F18BF9EEA445F00F0748021EA92
:1043E000045123EA0E0343F48013DCF1200E32D390
:1043F00022FA0CFE10EB0E0023FA0CFE41EB0E012C
:10440000CCF1200E03FA0EFE10EB0E00CCF1200EC4
:1044100051F10001B1F5801F32D201EB045112FAC3
:104420000EF2BDE8104058BF7047401C38BF5FEA2D
:10443000420218BF7047002814BF20F0010041F16C
:1044400000014FEA410313F5001F38BF7047A1F187
:10445000C04100F0B9BB012A43EB0302ACF1200CD0
:10446000DCF11F0E32BF4FF0000E23FA0CF310EBFD
:10447000030041EB0451B4EB115FD0D0A1EB045128
:1044800001F58011490801EB04515FEA30000ED3B9
:1044900050F1000038BF12FA0EFE08D1BDE81040FE
:1044A000C9E7401C38BF5FEA4202CAD1C3E7BDE892
:1044B00010404FEA410313F5001F38BF7047A1F1C8
:1044C000C04100F081BB9EEA445F08D011EA5E0F54
:1044D000BDE8104004BF01F0004100207047BDE876
:1044E000104070B500F022FB64FBBE3E0000E0FF10
:1044F000491058BFC1F140415B1058BFC3F1404360
:104500008B42EFF3008070472DE9C04130B4DFF8F3
:10451000A4C23CEA111418BF3CEA131400F0ED8069
:104520001CEA111481EA030544EAD57418BF1CEA99
:10453000131500F0C880A4EB050404F17F7404F5A2
:1045400000344FF0004545EAC12145EAC32341EA62
:10455000505143EA52534FEAC0204FEAC2229942D7
:1045600008BF904200F09D804FEA13650FF2441699
:10457000765D4FEA134506FB05F7C7F1807706FB2A
:1045800007F74FEAD737A7FB03687642A7FB06CEAB
:10459000C8F5803838BFA8F1010807FB08E6A6FB7C
:1045A000028C4FF0000EE6FB03CEDCF1000CCEF1E6
:1045B000004E38BFAEF1010EA6FB0C584FF00007BD
:1045C000E6FB0E87A1FB08C6A0FB07CE16EB0E0686
:1045D0004FF0000545F10005E1FB076515F1E04EE0
:1045E0007EBFA4F580345FEA46066D4116F1800770
:1045F00045F100054FEA172747EA05674FEA1525F9
:104600004FEA0666A6F1DE46B6F1805F20D938464D
:1046100005EBC47124F0010C01EB0C11BCF1FE6F31
:1046200002D8F0BCBDE8008124425CBF01F5801EC9
:104630009EEAC47F02D4F0BCBDE80081244200F1B0
:104640003980A1F1C041F0BCBDE8004100F0BCBA26
:104650004FEAD02040EA41504FEAD1214FEAD2221E
:1046600042EA43524FEAD323A7FB028607FB0366C5
:1046700005FB02661EEA0E0F58BFA6EB0056B6EB0E
:1046800000564FEA520E4EEAC37E18EB0E0E56EB62
:10469000530EBCD518EB02085E417F1C55F1000596
:1046A000B5E74FF480154FF000074FF000064FF0CC
:1046B0000008ACE701F1C04101F000414FF00000FB
:1046C000F0BCBDE800810CEA131511EA0C1F00D004
:1046D0000CE013EA0C1F00F026804FF0000081EA86
:1046E000030101F00041F0BCBDE80081F0BCBDE871
:1046F000004181EA030100F067BAF0BCBDE8004167
:1047000070B500F013FA00BF097EFC3E00F007B858
:104710004FF0000081EA030101F00041704781EA97
:10472000030100F051BAF0BCBDE8004122494FF04E
:1047300000007047FFFDFBF9F7F5F4F2F0EEEDEB4A
:10474000E9E8E6E4E3E1E0DEDDDBDAD8D7D5D4D38F
:10475000D1D0CFCDCCCBCAC8C7C6C5C4C2C1C0BFDB
:10476000BEBDBCBBBAB9B8B7B6B5B4B3B2B1B0AFE1
:10477000AEADACABAAA9A8A8A7A6A5A4A3A3A2A1C5
:10478000A09F9F9E9D9C9C9B9A9999989797969580
:1047900095949393929191908F8F8E8E8D8C8C8B1C
:1047A0008B8A8989888887878685858484838382A4
:1047B000828181800000FF070000F87F51EA030C2E
:1047C00017D41CF5801F58BFBCF5801F00F1068070
:1047D000994218BF704708BF9042704707D711F53C
:1047E000801F58BF13F5801F19D499427047894222
:1047F00070471CF5801F08D5BCF5801FF7D58B428C
:1048000018BF704708BF824270474FF4001C1CEB72
:10481000410F38BF1CEB430F01D28B42704770B57C
:1048200000F084F9922449004FF000514FF080537A
:10483000FFF75EBE4FEA41034FEA5353A3F580638F
:10484000D3F11E03C8BFD3F1210C0CDD4FF00042A1
:1048500042EAC12242EA505232FA03FC8CEAE17C7D
:10486000ACEBE1707047102BC4BF0020704703F51C
:10487000787CBCF1FF3F04D06FF0004282EA210057
:10488000704770B500F052F94992248000207047BB
:10489000F2E710F0004248BF4042B0FA80F310FA4D
:1048A00003F10AD0C3F11D0303F5806302EB035249
:1048B0004FEA415002EBD12170474FF000007047A2
:1048C000B0FA80F310FA03F10AD0C3F11D0303F527
:1048D00080634FEA03524FEA415002EBD121704707
:1048E0004FF000007047000051EA030C17D41CF58C
:1048F000801F58BFBCF5801F00F10680994218BF89
:10490000704708BF9042704707D711F5801F58BF06
:1049100013F5801F19D499427047894270471CF5DE
:10492000801F08D5BCF5801FF7D58B4218BF704794
:1049300008BF824270474FF4001C1CEB410F38BF88
:104940001CEB430F01D28B42704770B500F0EEF8BC
:10495000922449004FF080514FF00053FFF7C8BD3B
:1049600051EA030C17D41CF5801F58BFBCF5801FFB
:1049700000F10680994218BF704708BF9042704707
:1049800007D711F5801F58BF13F5801F19D499421E
:104990007047894270471CF5801F08D5BCF5801F01
:1049A000F7D58B4218BF704708BF824270474FF45B
:1049B000001C1CEB410F38BF1CEB430F01D28B4294
:1049C000704770B500F0B2F8922449004FF00051E2
:1049D0004FF08053FFF78CBD70B5DFF848C11CEA7B
:1049E000111E1EBF1CEA13159EEA0C0F95EA0C0F50
:1049F00000F06F8081EA03044EEAD47EAE4421EADF
:104A00004C1123EA4C1341F4801143F48013AEF1AE
:104A10007F7EA1FB024CA0FB0365361955EB0C050C
:104A2000A1FB034C4CF10003A0FB021C16EB0C068F
:104A3000654153F10003094218BF46F0010613F423
:104A4000007F0BD14FEA03314FEA053041EA15519F
:104A500040EA165034036FF003020AE04FEAC32124
:104A60004FEAC52041EA555140EA5650F4026FF032
:104A7000020202EB2E4201EB025585EACE710AD00A
:104A80005FEA440C18BF24F0004450F1000041F1EB
:104A9000000120EAD47040F2FE7C624500D270BD75
:104AA000A84214BF4FF080444FF04044002E08BF8E
:104AB0000024BEF1806FA8BFA1F1C041BDE87040E5
:104AC00080F2828001F1C04101F000414FF000000E
:104AD00070470CEA13159EEA0C0F18BF95EA0C0FED
:104AE00006D081EA030E4FF000000EF0004170BDC9
:104AF00000F01CF88900013E00F007B800F009B88A
:104B00004FEA430C5FEA5C5C08D081EA030100F0E5
:104B10005BB84FEA410C5FEA5C5CF6D102494FF0AA
:104B2000000070470000FF070000F87F0EF1020E42
:104B30002EF0030E5EF8046B364205D4012A43EBD7
:104B4000030515F5001F12D8012841EB010C1CF5D7
:104B5000001F0CD80ED14FEAD17C0CEB4C0C0CF1A1
:104B6000020C15F5001F08BF4CEBD37C04E04FF09E
:104B7000080C01E04FEAD37C0CEB4C0526FA05F655
:104B800006F00706B6F1040C06D20EEB860CBDE863
:104B900070404CF0010C6047DFE80CF0090B02029A
:104BA0004FF00041A1F500214FF0000070BD194603
:104BB0001046012851EB010418BFD4F5001484BF3E
:104BC000002001F0004170BD0808A0F500114FEA77
:104BD0003101704710B591EA030F48BF83F00043DD
:104BE0003FF5E6AB841A71EB030C07D28CF0004C56
:104BF000121943EB0C03001B61EB0C014FEA11543B
:104C0000A4EB135CDFF8A4E11EEA430F18BF9EEA91
:104C1000445F00F0B48021EA045123EA6E0352425B
:104C2000C3EB6E0338BF5B1EDCF1200E25D322FAE6
:104C30000CFE10EB0E0043FA0CFE41EB0E01CCF122
:104C4000200E03FA0EFE10EB0E00CCF1200E51F1F7
:104C5000000129D401EB045112FA0EF2BDE8104014
:104C600058BF7047401C1CBFB2F1004F704700286E
:104C70000CBF491C20F00100704712EB020E43EB01
:104C8000030218BF4FF0010E4EEA4202ACF1200CB5
:104C9000DCF11E0E56D943FA0CFE10EB0E00CCF1DF
:104CA0001E0E51F1FF31D5D50EF1010E12FA0EFE96
:104CB000404141EB010101EB445C5FEA5C5C10D9CF
:104CC00001EB045110EBDE7038BFBEF1004FBDE8C0
:104CD000104018BF704700280CBF491C20F001008D
:104CE000704734D24FEAD42C24F4006411F500113B
:104CF0001BD0B1FA81F20B3AA41AA41ED2F1200300
:104D0000914030FA03F31943904001EBCC7101EB71
:104D10000451002CBDE81040A8BF704701F1C0410C
:104D200001F000414FF000007047B0FA80F310FA34
:104D300003F102D1BDE810407047E41A173C480562
:104D4000C90AE2E701EB0451BDE810407047491081
:104D50004FEA300001EB0451BDE8104002E04FF093
:104D6000000170474A0008BF0042F8D0B2F5001FAA
:104D700028BF704701F000414FF0000070479EEAE5
:104D8000445F07D011EA5E0FBDE8104004BF002168
:104D900000207047BDE8104070B5FFF7C7FE00BFA8
:104DA00040DFF63E104683F0004170470000E0FF10
:104DB00043004FEAD30C4FEA3C0C43401FBF40076F
:104DC0000CF1605113F0FE4F70471CF0006F03D1DF
:104DD0000CF00041002070470CF0004343EA507093
:104DE00040EACC0010B500F0F8FA00BF00000092D5
:104DF0004FEA0001FFF7E8BE4FF00041A1F50021A6
:104E00004FF000007047000090EA010F48BF81F0AA
:104E1000004100F13483421A3CBF801A89184FEADE
:104E2000D052A2EBD1534FF07F4C1CEA410F18BF78
:104E30009CEA026F00F03B804FF0004C4CEA0020EF
:104E40004CEA012121FA03FC10EB0C0C1ED202F1FA
:104E5000FF325FEA1C2040EBC25038BF70471CF0A5
:104E60007F0F4FEA400C18BFBCF17F4F38BF70472F
:104E7000C3F12003994008BF20F00100BCF17F4F2F
:104E800038BF7047A0F1C04000F0EDBA4FEA3C00D7
:104E9000000A40EBC25028BF1CF0FF0F4FEA400C45
:104EA000E6D018BFBCF17F4F38BF7047EAE79CEAF5
:104EB000026F05D010EA5C0F08BF00F00040704799
:104EC00010B500F08AFA00BF64FBBE3E10B5FFF7D4
:104ED00075FC0CBF0120002010BD10B5FFF76EFC63
:104EE00014BF0120002010BD10B5FFF7FDFC8CBFE2
:104EF0000120002010BD10B5FFF7F6FC2CBF0120EB
:104F0000002010BD10B5FFF72BFD94BF012000203D
:104F100010BD10B5FFF724FD34BF0120002010BDE7
:104F200010B500F0F5F80CBF0120002010BD10B541
:104F300000F0EEF814BF0120002010BD10B500F005
:104F400063F98CBF0120002010BD10B500F05CF9A2
:104F50002CBF0120002010BD10B500F089F994BFCE
:104F60000120002010BD10B500F082F934BF0120EF
:104F7000002010BD401058BFC0F14040491058BF3C
:104F8000C1F140418142EFF3008070474FF47F0C44
:104F90001CEAD0121EBF1CEAD11392EA0C0F93EA4E
:104FA0000C0F00F0858090EA010F48BF42F4807238
:104FB00040F4000C41F400002CF07F4120F07F40D1
:104FC00000B5A2EB030281420FF2081CACEB504E7D
:104FD0009EF800E0C0F100004FEA4E0E00FB0EFC10
:104FE00038BF49004FEA2C1C0CFB0EF34FEACE1ED3
:104FF0000EEB635E4FEA112C0EFB0CFC4FEAC12155
:105000004FEA1C5300FB031102F5FA024FEA112C80
:105010000EFB0CFC4FEA01314FEADC4C00FB0C119B
:1050200042EB2242C14228BF09184CEB03335DF822
:1050300004EB10EB410143EBC250B2F57C0F38BFDB
:10504000704729D512F0F00F1CBF00F1C04000F0EE
:1050500000407047008182838485868788898B8C95
:105060008D8E8F919293959697999A9C9D9FA0A2D1
:10507000A3A5A7A8AAACAEB0B2B3B5B7B9BCBEC021
:10508000C2C5C7C9CCCED1D4D7D9DCDFE2E6E9ECC2
:10509000F0F3F7FAFE0000004FEA400C0CF1807CC0
:1050A000BCF17E4F28BF7047B0F1C04000F0DBB9C3
:1050B0000CEAD11390EA010F48BF42F480726245B6
:1050C00038BF634507D213F47F0F16D080EA010082
:1050D00000F00040704710B500F07FF9097EFC3EFB
:1050E00000F005B880EA010000F00040704780EA57
:1050F000010000F0004000F0B6B912F47F0F04BFC9
:105100000248704780EA010000F0ADB90000C07F9E
:1051100050EA010C00F113801CF5000F58BFBCF5DC
:10512000000F01D48842704707D710F5000F58BF11
:1051300011F5000F15D488427047894270471CF55D
:10514000000F04D5BCF5000FF7D5814270474FF032
:10515000807C1CEB400F38BF1CEB410F01D2814219
:10516000704710B500F039F9922449004FF0005013
:105170004FF08051FFF7FEBE41000B0ED3F19E02AF
:1051800008D950F400034FEA032323FA02F048BF82
:105190004042704710B500F020F900BF49922480CA
:1051A000002070476FF0004282EA20007047000044
:1051B00010F0004148BF4042B0FA80F310FA03F209
:1051C000C3F19D030BD051EAC35101EB12205306EA
:1051D00038BF704700F1010008BF20F001007047A0
:1051E000B0FA80F310FA03F2C3F19D030AD0D90597
:1051F00001EB1220530638BF704700F1010008BFD1
:1052000020F001007047000050EA010C00F113800B
:105210001CF5000F58BFBCF5000F01D48842704741
:1052200007D710F5000F58BF11F5000F15D48842AD
:105230007047894270471CF5000F04D5BCF5000F7C
:10524000F7D5814270474FF0807C1CEB400F38BF90
:105250001CEB410F01D28142704710B500F0BDF840
:10526000922449004FF080504FF00051FFF782BE6A
:1052700050EA010C00F113801CF5000F58BFBCF57B
:10528000000F01D48842704707D710F5000F58BFB0
:1052900011F5000F15D488427047894270471CF5FC
:1052A000000F04D5BCF5000FF7D5814270474FF0D1
:1052B000807C1CEB400F38BF1CEB410F01D28142B8
:1052C000704710B500F089F8922449004FF0005063
:1052D0004FF08051FFF74EBE4FF47F0C1CEAD01206
:1052E0001EBF1CEAD11392EA0C0F93EA0C0F00F0D8
:1052F000478090EA010F48BF42F480724FF0004CA3
:105300004CEA00204CEA012102EB0302A0FB01134E
:10531000A2F50002002918BF43F001035B0028BF7B
:105320004FEA330342EB22425FEA132C4CEBC250AC
:105330002EBFBCEB436FB2F57C0F70474FEA036C96
:10534000BCF1004F08BF20F00100B2F57C0F38BF60
:1053500070470BD582F0FF0212F5803FC8BF70473F
:1053600000F1C040D8BF00F00040704700F5000CCD
:105370005FEA4C0C48BF7047B0F1C04000F073B812
:105380000CEAD11390EA010F48BF42F480726245E3
:1053900038BF634504D280EA010000F00040704746
:1053A00010B500F01AF800BF8900013E00F007B800
:1053B00000F009B85FEA410C5FEA1C6C08D080EA93
:1053C000010000F050B85FEA400C5FEA1C6CF6D1B7
:1053D0004FF00040A0F5800070470EF1020E2EF055
:1053E000030E5EF8044B244204D44FEA4102B2F1AA
:1053F0007F4F11D84FEA4003B3F17F4F0CD80ED145
:105400004FEAD07C0CEB4C0C0CF1020CB2F17F4F4C
:1054100008BF4CEBD17C04E04FF0080C01E04FEAF0
:10542000D17C0CEB4C0324FA03F404F00704B4F130
:10543000040C06D20EEB840CBDE810404CF0010CBD
:105440006047DFE80CF0070802024FF00040A0F5CB
:10545000800010BD0846420018BFD2F1807288BF9C
:1054600000F0004010BDFF2141EAD050C005704758
:1054700090EA010F48BF81F000413FF5CCAC421AE1
:1054800004D882F00042A0EB020011444FEAD0524F
:10549000A2EBD1534FF07F4C1CEA410F18BF9CEA9E
:1054A000026F4AD04FF0004C4CEA00204CEA012138
:1054B00021FA03FCB0EB0C0C0FD412F0FE0F36D027
:1054C0005FEA4C001DD5001240EBC25038BF704758
:1054D0001CF03F0F18BF70470BE05FEA1C20A2F1E1
:1054E000010240EBC25038BF70471CF07F0F18BF5D
:1054F0007047C3F12003994014BF401E20F0010003
:1055000070474FEA1223800808BF7047B0FA80FC4A
:10551000A2EB0C02CCF1280C60FA0CF093EA122FEB
:1055200004BF00EBC25070474FEAC3707047130AC4
:105530005FEADC1008BF7047F6E79CEA026F04D010
:1055400010EA5C0F08BF0020704710B5FFF745FF59
:1055500040DFF63E81F0004070470000FFFFFEFF95
:10556000000002000100110A120A130A140A110AAB
:10557000160A0000000001020304000305040102F2
:1055800006000000000080BF82EC6FBF4FD160BFFB
:105590006E9652BFE02645BF267038BFEB612CBF28
:1055A000AFED20BF8A0616BFF6A00BBF9EB201BFAB
:1055B0007264F0BED02EDEBE32B5CCBEE2E9BBBE18
:1055C00068C0ABBE6A2D9CBE8B268DBE9C447DBE42
:1055D000043061BE52FF45BECFA32BBEE70F12BE03
:1055E0001E6EF2BD521BC2BDDB1193BD617B4ABD75
:1055F000B430E2BCD9BECEBB639A6D3C67C10E3DF0
:105600000A55603D211E983D1848BF3D41B4E53D17
:10561000E4B6053E9C3F183E47792A3EA1683C3ED1
:1056200029124E3E257A5F3EA7A4703EC9CA803E2D
:105630004F28893EAE6C913E9A99993EB7B0A13EF3
:105640009CB3A93ECEA3B13EC982B93EF951C13E39
:10565000C212C93E7FC6D03E816ED83E130CE03EDA
:1056600076A0E73EE82CEF3EA2B2F63ED832FE3EF0
:105670005CD7023FBA93063F194F0A3F110A0E3F0B
:1056800035C5113F1C81153F593E193F85FD1C3F13
:1056900036BF203F0684243F904C283F71192C3F91
:1056A0004AEB2F3FBEC2333F75A0373F1A853B3FC1
:1056B0005C713F3FF065433F9263473F016B4B3F57
:1056C000067D4F3F709A533F15C4573FD6FA5B3F54
:1056D0009D3F603F5D93643F17F7683FD86B6D3F18
:1056E000B8F2713FE08C763F8A3B7B3F0000803F01
:1056F000CF6D823FECE7843F1A6F873F2B048A3FD0
:10570000FDA78C3F7C5B8F3FA51F923F88F5943FA0
:1057100047DE973F18DB9A3F4BED9D3F4816A13F70
:105720009557A43FD6B2A73FD429AB3F7DBEAE3F2D
:10573000EC72B23F6A49B63F7744BA3FD066BE3F8B
:1057400076B3C23FB52DC73F30D9CB3FECB9D03F80
:105750005DD4D53F772DDB3FBDCAE03F5AB2E63F6F
:1057600038EBEC3F207DF33FDE70FA3F37E8004036
:1057700094D30440090109400D780D404341124083
:10578000B166174010F41C4029F722404D80294093
:10579000F5A230408D76384085174140B7A84A4081
:1057A00055555540965361406CE86E40ED6C7E4017
:1057B0001E2B8840C4A0924061039F4076EBAD4011
:1057C000A037C040253AD740420FF54030A70E41E0
:1057D000C14E2B4184695741B0119241148AE54171
:1057E00022E98942907E1EC384DE10C2EBD4A1C19F
:1057F0004DCE5EC179D028C12A2A07C1C957E0C061
:105800004EE9BEC0467FA5C0A68391C0786181C025
:10581000382668C00CD051C084C93EC0C5602EC0B7
:10582000731220C06D7B13C07C4F08C024A6FCBF40
:10583000F1ADEABF886ADABF539ECBBFC316BEBFC5
:10584000F9A9B1BFF834A6BF4A9A9BBFF3C091BF74
:10585000A09388BF000080BF785800080000002097
:1058600010000000A4010008885800081000002063
:10587000580A0000C001000800A24A0400002042AB
:085880000100D007E80320201D
:040000050800016985
:00000001FF
